:020000040800F2
:10000000F0050020D50000086F11000869110008F4
:1000100000000000000000000000000000000000E0
:10002000000000000000000000000000BD140008F7
:100030004D04000800000000B5110008C9140008B4
:10004000E9000008E9000008E9000008E9000008EC
:10005000E9000008E9000008E9000008E9000008DC
:10006000E9000008E9000008E9000008E9000008CC
:10007000E9000008E900000800000000E9000008AD
:1000800000000000E900000800000000000000007F
:10009000E900000800000000E9000008E90000088D
:1000A000E9000008E9000008E9000008E90000088C
:1000B000E9000008E9000008E9000008E90000087C
:1000C0000348854600F02CF800480047B12A000894
:1000D000F00500200548804705480047FEE7FEE799
:1000E000FEE7FEE7FEE7FEE7FEE70000D5140008A6
:1000F000C100000830B50B46014600202022012433
:1001000009E00D46D5409D4205D31D469540491B4B
:100110002546954040191546521E002DF1DC30BD94
:10012000064C0125064E05E0E36807CC2B430C3C4A
:1001300098471034B442F7D3FFF7C6FF1C460008B7
:100140003C460008F8B5094D0746002468681123AD
:100150008668AB2221462046B047054E6968F8B252
:1001600049688847641CB442F8D3F8BDF800002001
:10017000180C0000F8B5203A104FD3B23A68D48872
:1001800096882546754312685D43AA1800920A199D
:10019000521E93B27F6800258219521EBF6892B228
:1001A000B8477443054E05E0716800984968405DA2
:1001B00088476D1CA542F7D3F8BD0000F800002069
:1001C000FFB50546002681B014463746104600E0CC
:1001D0007F1C0178401C0029FAD100F0B3F81E49B9
:1001E000096889880091FFF785FF0499012902D0E9
:1001F00002290BD105E00099C01B48434008401973
:1002000003E00099C01B4843401B85B2124F00F029
:1002100099F801463868808802467243891A89B283
:1002200081420DD301200CE028460299FFF7A2FF7E
:100230003868761C8088B6B2401985B2641CE6E73F
:1002400000202278002A01D0012100E0002108428C
:10025000EAD105B0F0BD0000F8000020F8B5094E65
:1002600015467368002442199F6892B20B46B8473E
:1002700004E0706841683F208847641CAC42F8D3B2
:10028000F8BD0000F8000020FFB581B00298910889
:1002900008181E46401E83B2019817468019401E5A
:1002A0000F4C82B26068029985680198A84760681F
:1002B000C569002D06D00A98009033463A46029947
:1002C0000198A84700F044F885B200F03BF882B2EC
:1002D0006068002184682B460846A04705B0F0BD41
:1002E000F8000020F8B51D4614460E460746FFF7F5
:1002F000B5FF601C82B2701981B23846FFF7AEFFBD
:100300002A463146384600F007F8381980B22A46A6
:10031000314600F001F8F8BDF8B5154600244A1939
:10032000074E93B2726897680246B84704E0706857
:10033000416800208847641CAC42F8D3F8BD000037
:10034000F80000200148406840690047F80000209C
:100350000148406880690047F800002010B508484F
:100360000446083C20600748606000688047FF2022
:10037000FFF7E8FE204610302060002010BD00008E
:1003800000010020D800002070B50B484068C0680C
:100390008047FF24013405252D072146284600F01B
:1003A000B5F90028F9D101220421044800F0B3F97D
:1003B0000A2000F04CF870BDF80000200004005046
:1003C000F0B50F4A02230121D46A85B0002815D068
:1003D0000C43D4620B4D44002A5B01910A4F0291F9
:1003E000860003930092B859694600F0D5F8295B5E
:1003F000B859002200F08FF905B0F0BD1C43E8E7C2
:10040000001002409C2D0008D000002010B5054AC5
:100410004100515A044A80001058002200F07BF934
:1004200010BD00009C2D0008D000002010B5054A2A
:100430004100515A044A80001058012200F06BF923
:1004400010BD00009C2D0008D0000020704710B5A2
:1004500000F096F810BD0000F0B52B4885B0C16AD9
:1004600001221143C162C16A02242143C162C16AEF
:100470002143C162C16A1143C162C16A2143C162A1
:1004800003200390D50300260520694602960095B7
:100490000192000700F080F8A002009069461B4816
:1004A00000F07AF8042000906946184800F074F8CB
:1004B000670269461548009700F06EF8E001009069
:1004C0000520694601960294000700F065F80022B5
:1004D00039460E4800F01FF9052000222946000782
:1004E00000F019F9052001222946000700F013F950
:1004F00001220421054800F00EF90A2000F040F81E
:1005000000F086FF05B0F0BD00100240000400506E
:1005100070B5012505260446ED033607002229465D
:10052000304600F0F8F80122D102064800F0F3F856
:10053000E0B200F0B3FF01222946304600F0EBF8AC
:1005400070BD00000004005070B50124052506466A
:10055000E4032D0700222146284600F0DCF80022A3
:100560002111064800F0D7F8304600F097FF01222D
:100570002146284600F0CFF870BD0000000400506E
:1005800031B500F0CFF8044600F0CCF80099001B1C
:100590008842F9D338BD0000F8B500220124254671
:1005A0000B6895402B40AB426FD14E68022E01D0B4
:1005B000122E14D1D608B60036180096366A5707A0
:1005C000B446FE0E0F27B646B7406646BE43B44655
:1005D0000F697646B74066463743009E37624E68DD
:1005E000012E05D0022E03D0112E01D0122E16D1CD
:1005F00087680326BC465700BE46BE406746B743E1
:10060000BC46CE687746BE4067463E438660466835
:10061000AE430D79ED06ED0F954035434560076813
:1006200056000325B540AC46AF430D79AD07AD0F7D
:10063000B5403D430560C7686546AF438D68B5402A
:100640003D43C5604D68ED004CD5294D6E6B26438A
:100650006E639608274DB6007519AF68AC469507CE
:100660002E0F0F25ED43B5403D4005273F07B8420B
:1006700001D1002715E0204FB84201D1012710E039
:100680001E4FB84202D102270BE02BE01C4FB842AC
:1006900001D1032705E01B4FB84201D1042700E038
:1006A0000527B7402F436546AF60174D2E684F684A
:1006B0009E43FF0300D51E432E606E684F689E4325
:1006C000BF0300D51E436E60AE684F689E43FF02B5
:1006D00000D51E43AE60EE684F689E43BF0200D552
:1006E0001E43EE60521C102A00D258E7F8BD0000ED
:1006F00000100240000001400004005000080050BB
:10070000000C0050001C005000040140006908402B
:1007100000D001207047002A01D0816170478162BA
:10072000704700000148006870470000AC000020DE
:1007300002480168491C016070470000AC000020BD
:1007400010B5084801684022114301600168022287
:1007500011430160032000F007F800F017F80020B3
:1007600010BD00000020024010B5044600F05EF904
:100770007D21C900FFF7BEFC00F08CFC0022214661
:10078000501E00F04DF8002010BD0000F0B52248CA
:1007900085B0016B0122120411430163C16A012576
:1007A0002943C162C16A02263143C162122001900D
:1007B00088200024009003270520029404970394C6
:1007C00069460007FFF7E8FE694614480096FFF700
:1007D000E3FE4420009005200294694604970196A8
:1007E00003940007FFF7D8FE69460C480095FFF711
:1007F000D3FE10200090029403946946019504945E
:100800000648FFF7C9FE2020009005206946000732
:10081000FFF7C2FE05B0F0BD00100240000400501A
:1008200010B500F0A5FC10BDF8B505467C480E4695
:100830000068F021C007C00F7A4CB04268D27848F7
:10084000026852085200324302600068C007C00FBD
:10085000B0427DD12878800704D5E0688843A96834
:100860000843E0602878C0072FD06868022818D0B5
:10087000002819D02168032819D04907002967DA10
:10088000E168890889000143E160FFF74BFF0646F4
:100890006868022813D003281ED0634F002827D091
:1008A00030E021688903E9E721688905E6E78901E5
:1008B000E4E7FFF737FF801BB84201D981E05A4FC8
:1008C000E0680007800F0228F3D18EE0FFF72AFFCF
:1008D000801BB84201D974E0534FE0680007800FD5
:1008E0000328F3D181E0FFF71DFF801BB84268D8D1
:1008F000E0680007800FF6D177E0FFF713FF801B59
:10090000B8425ED8E0680007800F0128F5D16CE09E
:100910002878800704D5E0688843A9680843E06028
:100920002878C00754D06868022819D000281AD047
:10093000216803281AD04907002954DAE168890898
:1009400089000143E160FFF7EDFE0746686800E0BB
:1009500049E0022812D003281CD0002826D032E01B
:1009600021688903E8E721688905E5E78901E3E76C
:10097000FFF7D8FEC11B2C48814222D8E06800074F
:10098000800F0228F4D123E0FFF7CCFEC11B2648DC
:10099000814216D8E0680007800F0328F4D117E0E1
:1009A000FFF7C0FEC11B204881420AD8E06800075B
:1009B000800FF5D10CE0FFF7B5FEC11B1A4881424C
:1009C00001D90320F8BDE0680007800F0128F2D1AB
:1009D0001348016849084900314301600068C007B5
:1009E000C00FB04201D00120F8BD2878400706D5DD
:1009F000E068072109028843E9680843E060287835
:100A0000000707D5E0680721C90288432969C900A2
:100A10000843E0600320FFF7A7FE0020F8BD0000B8
:100A200000200240001002408813000010B500F0C2
:100A300011F80549C968054A0906090F515CC84003
:100A40000349086010BD000000100240B9000020FA
:100A50004C00002010B5174A506817490004400F99
:100A600080000858D1680C23194019D0042918D0E7
:100A700008291DD00C2913D1D068D16880020F4BF2
:100A8000000F185C0902D268890F01231B04491C5E
:100A90001A4201D10A4A00E00A4A5043FFF72AFBF2
:100AA00010BD1068C00601D5074810BD044810BD30
:100AB000044810BD001002407C2D0008B00000204A
:100AC0000024F40000127A0000093D00F8B5044645
:100AD0000078E84DC0074CD0E8680007800F022876
:100AE00007D0E8680007800F03280BD1E868C0032F
:100AF00008D5286880033CD5012061680004814244
:100B000072D136E029680520000481432960FFF78F
:100B100009FE0746D84E04E0FFF704FEC01BB042B2
:100B20007DD828688003F7D4286805210904884304
:100B300061680843286001206168000481420CD18B
:100B4000FFF7F0FD074604E0FFF7ECFDC01BB042E5
:100B5000E6D828688003F7D50BE0FFF7E3FD0746EA
:100B600004E0FFF7DFFDC01BB042D9D8286880033E
:100B7000F7D42078800740D5E8681F270007800F4A
:100B80003F02012807D0E8680007800F032809D139
:100B9000E868C00306D42868400717D5E068012834
:100BA000AED113E0E1680920002916D02A688243FB
:100BB0000A432A60FFF7B6FD064604E0FFF7B2FDE0
:100BC000801B6428ACD828684007F7D5686821697D
:100BD000B8430902084368600FE02968814329602F
:100BE000FFF7A0FD064605E042E1FFF79BFD801BF5
:100BF000642895D828684007F7D420789F4FC0060E
:100C00003AD5E8680007800F0AD0E0690028286814
:100C100024D038432860FFF785FD06460CE0BFE08E
:100C2000286880050BD5E0690128B9D107E0FFF7F6
:100C300079FD801B64288BD828688005F7D5686803
:100C4000072149038843616A084368606868218C0A
:100C50000002000A0906084368600DE0B8432860F6
:100C6000FFF760FD064604E0FFF75CFD801B64288B
:100C7000A8D828688005F7D42078814E000724D5AD
:100C800060690028306910D0012108433061FFF706
:100C900049FD009005E0FFF745FD0099401A6428E2
:100CA0007ED830698007F6D50FE0400840003061FB
:100CB000FFF738FD009005E0FFF734FD0099401A7A
:100CC00064286DD830698007F6D42078800632D544
:100CD000A0696C4A002818D0A96801200143A960C6
:100CE000696B01436963106A674908431062FFF743
:100CF00019FD009005E0FFF715FD0099401A6428E2
:100D00004ED8A8688007F6D515E0A86840084000CE
:100D1000A860106A5C49C94308401062FFF702FDF1
:100D2000009005E0FFF7FEFC0099401A642837D8D0
:100D3000A8688007F6D42078400751D5A86B012118
:100D400009070843A86351480168821511430160EF
:100D5000FFF7E8FC074604E0FFF7E4FCC01B64284B
:100D60007FD84A480068C005F6D5316905200002E1
:100D700081433161FFF7D6FC3F4F009005E0FFF75C
:100D8000D1FC0099401AB8426BD830698005F6D47E
:100D90003069052109028843A1680843306100E0F9
:100DA0005FE0A168C81FF93803D0FFF7BBFC0090D3
:100DB00013E0FFF7B7FC009005E0FFF7B3FC0099E4
:100DC000401AB8424DD830698005F6D508E0FFF7E3
:100DD000A9FC0099401AB84243D830698005F6D47E
:100DE000A06A002842D0E9680907890F03293FD08B
:100DF000012636060228286805D0B0432860FFF790
:100E000091FC04462FE0B0432860FFF78BFC0746B7
:100E100004E0FFF787FCC01B642822D82868800103
:100E2000F7D4616B206BEA680843E16AFD231B0479
:100E30009A4311430843E860286830432860FFF76D
:100E400071FC044604E0FFF76DFC001B642808D821
:100E500028688001F7D509E0FFF764FC001B6428CF
:100E600001D90320F8BD28688001F5D40020F8BD21
:100E70000120F8BD001002408813000000010000AE
:100E800040100240000001400120000000700040BE
:100E900010B5002810D00222014640310C464A7499
:100EA00001680A6840239A430A6000F04BF800206A
:100EB000A0746074207410BD012010BD4030407CCF
:100EC000704770B5040005D025464035687C002881
:100ED00002D004E0012070BD204600F034F802206A
:100EE000687420680168402291430160A1686068CD
:100EF00022690843E16811430843616901220843FC
:100F0000A169520211400843E1690843216A08437C
:100F1000A16A084321680860A0690421000C084008
:100F2000616A0843216848602168E06A08612068B6
:100F3000C16992009143C1610020A87401206874C6
:100F4000002070BD70477047FFB505460446403528
:100F5000687C81B0012871D100293BD0002A39D0AA
:100F6000287C01286AD00120287412206874002788
:100F7000AF742163A286E286E764A764A787E78748
:100F80000126A06A7603B04207D120680168B14308
:100F9000016020680168314301600121A068C90334
:100FA000884205D120680168012292031143016043
:100FB00020680168490603D401684022114301609A
:100FC000E0680028606808D0002820D0E08E012862
:100FD0001DD026E0012005B0F0BD002802D0E08E33
:100FE000012808D1206B411C216321680078C8606A
:100FF000E08E401EE0860004000C20D0002202217A
:101000002046049B00F0A0F9002815D1EAE7206BE8
:1010100021680088C860206B801C2063E08E401E21
:10102000E0860004000C0AD0002202212046049B26
:1010300000F08AF90028EAD00320CCE728E0A06A73
:10104000B04205D1206801680122120311430160FA
:10105000002202212046049B00F076F92026002879
:1010600007D1012280212046049B00F06DF9002861
:1010700003D0A87C3043A874DEE7A068002802D122
:101080002068C1688068012068742F740020A2E77E
:101090000220A0E7094910B5401E884201D901206D
:1010A00010BD074C60610321081F00F061F80020AB
:1010B000A06107202061002010BD0000FFFFFF009D
:1010C00000E000E070B5040023D002202546203562
:1010D0002877204600F047F8206801260660A168BE
:1010E0006068228A08436169520411430843A16978
:1010F0000843E1690843216A0843616A0843A16A19
:10110000084321680A6810430860E068012802D09B
:1011100007E0012070BD206801680122120411431C
:101120000160616B206B0843A16B08432168C043D9
:101130000861616B206B0843216888622168A06B9D
:101140000862206B00F0F0F92168086320684168AC
:101150008908890041602068816803221143816009
:101160002E77002070BD7047FEE7704770477047CC
:101170008307FF22DB0E9A408907090E9940002859
:101180000BDA0007000F0838830808489B0018187E
:10119000C36993430B43C3617047830804489B00B2
:1011A0001B181868904308431860704700ED00E072
:1011B00000E400E070470000F8B5514D2868007861
:1011C0000A2801D0042878D10020FFF72FF9012048
:1011D000FFF71CF928684B4E8078341F04281CD276
:1011E0002068012819D0FF20FEF7ACFF012346A29A
:1011F0000A210020FEF7E4FF04238C2203210F20A4
:10120000FFF770F810222323032110460096FFF702
:101210003BF8FFF7B9F80120206028688078001FAC
:1012200004281CD22068022819D0FF20FEF78AFF6C
:10123000012339A20A210020FEF7C2FF04238C22D9
:1012400003210F20FFF74EF8232310220321322021
:101250000096FFF719F8FFF797F80220206028683A
:101260008078083804281CD22068032819D0FF2071
:10127000FEF768FF01232CA20A210020FEF7A0FF41
:1012800004238C2203210F20FFF72CF823231022A4
:10129000032155200096FEF7F7FFFFF775F80320AE
:1012A0002060286880780C281ED3206804281BD072
:1012B000FF20FEF747FF012300E015E01EA20A21F0
:1012C0000020FEF77DFF04238C2203210F20FFF76F
:1012D00009F823231022032178200096FEF7D4FF7B
:1012E000FFF752F80420206028680078022805D112
:1012F0000120FFF79BF80020FFF788F8F8BD0000F9
:101300003C2D000804000020545320506F73697472
:10131000696F6E203D203100545320506F73697403
:10132000696F6E203D203200545320506F736974F2
:10133000696F6E203D203300545320506F736974E1
:10134000696F6E203D203400F8B51D4616460F46E5
:101350000446FFF7E7F9314626464036009000295B
:101360001ED043E0681C1BD0002D05D0FFF7DAF932
:101370000099401AA84213D920684168E02291439D
:1013800041602068026840218A43026023E02168AE
:101390000A6882430A6021680A6802430A601FE003
:1013A0002068816838468843DCD124E0681C1DD061
:1013B000002D06D0FFF7B6F901460098081AA8429A
:1013C00014D920684268E0218A434260206801689D
:1013D0004022914301600120A16A40038142D6D09E
:1013E00001207074002030740320F8BD20688168EB
:1013F00038468843DAD00020F8BD000010B5034815
:10140000FFF746FD00F004F810BD00009C0100202D
:10141000F0B585B01D48FFF751FD002834D11B48B9
:101420001B490160FF2100240531846041601021C7
:10143000C460C16102250462012105614A0284621F
:10144000826141610722134E4462C262F06A2843FE
:10145000F0620820009003200F4F02910390019545
:10146000694604943846FFF797F8202000906946B3
:10147000029504943846FFF78FF8706BE902084331
:1014800070630248FFF71DFD05B0F0BD9C01002010
:1014900000300140001002400004005001B501235B
:1014A0001B03012269460448FFF74EFD002801D0C6
:1014B000FFF7A4FF08BD00009C010020704700E07A
:1014C000401E0028FCD1704710B5FFF731F901F03C
:1014D00083F910BD10480168821511430160C1688D
:1014E0000E4A1140C16001680D4A114001608168D7
:1014F000490849008160016801229204914301601A
:10150000C168FD2212049143C160002101610549B7
:10151000C003886070470000001002400C40FF8844
:10152000F6FFF6FE00ED00E070B5044600200F2542
:10153000014601238E002A46B240224202D01A46BA
:101540008A401043491C0829F4D370BD10B5084CDB
:101550000849606008480068FEF7CCFD7D21C9009D
:1015600048434821FEF7C6FD2061002010BD000061
:101570008401002040420F004C000020F0B50028FC
:1015800001D00220F0BD14490023486814C80B7232
:10159000124983688B62C3680B630023083815E027
:1015A00025880C2786687D43755DED06AD0F032DFC
:1015B00009D096680F6BB7430F63002D03D15568B0
:1015C0008E6AAE438E620C325B1CA41C85899D42E0
:1015D000E6D80020F0BD0000840100200040024059
:1015E000F7B586B00021039146494A681821414366
:1015F000551882CD083D0291002802D0022009B082
:10160000F0BD002678E03C880C20A96844430859C6
:10161000C206920F032A69D1012210430851029891
:10162000007800F0A5F8009020460A30AA6801462C
:101630000490105A019000985052334900980A883B
:10164000824205D9A868062201599143091D06E086
:1016500049888142A8680AD20159062211430151E2
:10166000A968002008340853022003903EE00019C6
:1016700000F08EF8002825D00798002807D0079A98
:101680000099019890470090AA6804995052A9685F
:10169000201D085A009900F065F8009000F060F8ED
:1016A0008007AA68410F1059062398430843105138
:1016B00008980028009801D008998847A96808343C
:1016C000085313E0A968201D085A009900F04AF851
:1016D0002146AA680831505200F042F8AA688007F3
:1016E00011590623400F9943014311510298761C6A
:1016F0000C30F6B2BF1C0290A889B04283D8039880
:101700007DE70000840100208800002010B5094C0E
:10171000A06803210843A06007480069FFF7CFFED7
:1017200020681021084320602068022108432060BF
:1017300010BD000000400240840100200749012044
:10174000CA68D20707D00868102290430860C868AA
:10175000800701D5022070470020704700400240FA
:1017600000207047401A00B27047401A80B270479C
:10177000082805D2034980004018406B80B27047AA
:101780000020704700400240012070470020704751
:101790000120704770470000F7B5002084B007466D
:1017A00004460191009006980126FF2801D9FF20E8
:1017B0000690049800250068029036E0029800F038
:1017C000A3FF1F48C1680978202905D0212903D02B
:1017D000222901D0232906D140690168097802290C
:1017E0001ED187898468002C02D00020421E15E09B
:1017F000002007B0F0BD0821615E002907D00099E4
:1018000003DA002903DC009205E0002901DA002652
:1018100001E001210091401CC0B20C34B842EAD36F
:10182000029808306D1CEDB2029004988088A8429E
:10183000C4D8002E02D006980190DAE70198D8E7C4
:101840008401002070B50446C0880021C207002A28
:1018500002D08006C00E02D0A17261722CE0A07A84
:101860000125002803D0607A00280DD017E0134826
:101870000369022293430361114B1B88A38103690F
:1018800013430361A57261722146FF200C31F530CC
:1018900000F04AFF00280DD0607A00280CD01422F6
:1018A0000A212046FFF778FF0146204600F00AF89B
:1018B000002070BD6572F2E7012070BD00E000E01D
:1018C00084010020F3B5002785B00D463C46029701
:1018D000FF2900D9FF250598FF21006800902846C0
:1018E0004840401C80B2039000203FE0009800F088
:1018F0000BFF2248C1680978202905D0212903D08F
:10190000222901D0232908D14069016809780229D8
:1019100026D1878984681A480290002C2CD0002692
:101920001CE00821615EA088FFF71FFF0102A0886C
:10193000A27900021018039A694350430818010A5B
:10194000A171000CA0802046FFF720FF012802D1E2
:10195000029900208847761CF6B20C34BE42E0D3D0
:101960000098083000900198401CC0B20190059882
:10197000818801988142B9D807B0F0BD8401002068
:1019800025250008F8B5A049A0484B6900229D68AC
:1019900042808280C280027042701A68802354683C
:1019A0009C4354604E69B389032B6BD3002222E021
:1019B0000821695E002900DA00210227C75FBC46C2
:1019C000614508DD8788C780674687804180017848
:1019D000417002700CE00427C75FB94203DDC78085
:1019E0008180427004E00627C75FB94200DDC180F4
:1019F000521CD2B20C359342DAD875680422E978C9
:101A0000825E4908491E91423CDCC1884788521ACF
:101A1000791A077840787B435B0040001818736997
:101A200089B21F5E308B92B24843738B80B28918A3
:101A30000093FEF75FFB002F02DD7900081802E03B
:101A400079424900081A704900B2CA681278202AFF
:101A500019D0212A17D0C0B232686D4B6D492604C7
:101A60006CD55678C7B2B74238D9BF1BFF2F35DACD
:101A70002F7BF619864218DDA87A8C438006800CED
:101A800004435460B5E0009A002801DD801A03E0A9
:101A9000FF2301339A1A101800B2002801DA00203F
:101AA000DAE7FF28D8DDFF20D6E70E26F441E41858
:101AB0001226554DF44154606E69A7043268BF0E7A
:101AC00022D176688C43B67AB606B60C344354609D
:101AD0006A6901251268ED03AC4354604A4CC71D86
:101AE0006669F83735686A78BA4273DD7668377B9D
:101AF000D219C71DF937BA4207DD68688843B17A41
:101B00008906890C0843686073E06A680E26F24112
:101B1000D2181223DA416A60656996042B68B60E02
:101B200067D18A436968897A8906890C0A435A60B1
:101B300061690123DB0309689A434AE05678C7B21A
:101B4000B7421FD2F71BFF2F1CDA2F7B3F18B7427B
:101B500092DC0E26F441E41812262B4DF441546019
:101B60006E69A7043268BF0E43D176688C43B67A9B
:101B7000B606B60C344354606A6901251268ED0359
:101B80002C435460204C666935686A78D71DF83755
:101B900087421FDA7668FF32377B01323F1897425F
:101BA000ABDC6A680E26F241D2181223DA416A6071
:101BB000656996042B68B60E1BD18A436968897AD9
:101BC0008906890C0A435A60616901230968DB03AD
:101BD0001A434A600C49C0B24A690824126850701E
:101BE0004A6953681268DB7AE31AD84093788342D3
:101BF00001D10220F8BD90704869802200684168D8
:101C0000114341600020F8BD84010020A0000020A5
:101C1000000000FC003F0000F8B500F061FB2D4C17
:101C20000028606903D000273E4685682DE04168A2
:101C30000068497AC17060690029006802D00E21ED
:101C40000170F8BD0D21FBE7698900910068C1783A
:101C50002148007981420AD128460099FFF794FD76
:101C6000002802D00098A8800CE0AE80F8BDA988BA
:101C70000098081880B2A8800099884202D2AE80ED
:101C80000D2022E07F1CFFB20C3560698189B942CA
:101C9000DAD80168C878002804D0401E0006000E7B
:101CA000C870E3D160690D4A80680021128907E09D
:101CB0008388D34083808671491C0681C9B20C3069
:101CC00063699B898B42F3D80220616909680870B7
:101CD000F8BD00008401002088000020A000002042
:101CE00010B50A48026902218A430261084A536911
:101CF00092781B6892065C68A409A401920E1443B2
:101D00005C6002690A43026110BD000000E000E06F
:101D10008401002030B500F0E3FA02250E4C0028C3
:101D200007D0606901214068007900F033FB00288A
:101D300003D060690068057030BD60690068C178D3
:101D4000002904D0491E0906090EC170F4D10020F3
:101D500000F0E8FB30BD00008401002030B500F049
:101D6000BFFA02251A4C00280FD060690121406893
:101D7000807800F0F9FA002860690AD040680021F4
:101D8000007800F0F1FA002811D060690068057051
:101D900030BD0168C878002804D0401E0006000E3F
:101DA000C870F5D161690A20096808700DE06069A2
:101DB000416800688979C17060690029006802D0B3
:101DC0000721017030BD06210170FFF789FF30BD8A
:101DD0008401002008B500F083FA184B002815D0C4
:101DE00000F0CAF96946087008785F210840694622
:101DF00008700878012815D0022818D0042818D0B7
:101E0000082818D0002000F08DFB08BD5869016833
:101E1000C878002804D0401E0006000EC870F4D117
:101E20000D2000E0022059690968087008BD0620ED
:101E3000F9E70A20F7E70C20F5E70000840100200D
:101E400030B500F04DFA0A251A4C00281BD0606905
:101E500001214068C07800F071FA002813D0606951
:101E600000214068407800F069FA002860690ED0CF
:101E700041680068097AC17060690029006816D05D
:101E80000421017030BD60690068057030BD0168D3
:101E9000C878002804D0401E0006000EC870F5D196
:101EA0006169062009680870FFF71AFF30BD02213A
:101EB000E7E700008401002030B500F011FA0225A8
:101EC0001A4C00280FD0606901214068807800F02A
:101ED0004BFA002860690AD040680021007800F0C1
:101EE00043FA002811D060690068057030BD416870
:101EF0000068C979C17060690029006802D00B21AF
:101F0000017030BD0A2101700DE060690168C87878
:101F1000002804D0401E0006000EC870F1D161698F
:101F2000062009680870FFF7DBFE30BD8401002041
:101F300030B500F0D5F90C251A4C00281BD060698B
:101F400001214068C07800F0F9F9002813D06069D9
:101F500000214068407800F0F1F9002860690ED057
:101F600041680068097AC17060690029006816D06C
:101F70000521017030BD60690068057030BD0168E1
:101F8000C878002804D0401E0006000EC870F5D1A5
:101F90006169062009680870FFF7A2FE30BD0221C2
:101FA000E7E700008401002030B500F099F90A2528
:101FB000134C00281ED0606901214068C07800F0F1
:101FC000BDF9002816D0606900214068407800F013
:101FD000B5F9002812D060690068C178002904D0E2
:101FE000491E0906090EC17003D102206169096802
:101FF000087030BD60690068057030BD0620F5E7E7
:102000008401002030B500F06BF906250E4C002845
:1020100016D0606900214068407800F08FF90028F0
:102020000ED060690168C878002804D0401E000600
:10203000000EC87003D1616902200968087030BDC4
:1020400060690068057030BD8401002030B500F083
:1020500047F90C25134C00281ED060690121406807
:10206000C07800F06BF9002816D060690021406844
:10207000407800F063F9002812D060690068C178E8
:10208000002904D0491E0906090EC17003D102209F
:1020900061690968087030BD60690068057030BD0D
:1020A0000620F5E78401002038B500F019F9304C1E
:1020B000002860691AD040680121C07800F03EF91C
:1020C00000281FD0606900214068407800F036F990
:1020D00000283CD0616948680968007AC870616965
:1020E0000028096842D00420087038BD41680068A3
:1020F000497AC17060690029006801D0112130E07F
:102100000D212EE0E0681B4D0078202819D02228F0
:1021100017D0E86880688047002815D0A879811E0C
:102120003E29E2D261696A46096809798906890E01
:102130001170694600F024FB0028D6D100F0F2F9B6
:1021400038BD6069006AE5E7FFF7CAFD38BD606920
:10215000416800688979C17060690029006802D00F
:102160000821017038BD06210170EDE70220BBE7B0
:10217000840100208800002007490020CA681278E6
:10218000202A01D0222A05D14869C1690068007857
:10219000C000085C704700008401002010B51A4898
:1021A0000A22416949680A70436905215B685970D0
:1021B000436950215B68997044694B236468E370FC
:1021C00043695B6819714169032349684B7144692C
:1021D00002216468A17144696468E17144696468BA
:1021E0002172416949684B72436904215B68D97265
:1021F000416949680A734069012140688172002081
:1022000000F090F910BD00008401002070B500F0CE
:102210007DF8114C002804D060690068007813280C
:1022200018D1606901680D78E1680978202901D02A
:10223000222904D1C169E800001D0858804760695F
:10224000402100680278AA42426801D18A4300E036
:102250000A43426070BD00008401002010B5084AA6
:10226000506981680020034604E08B80401C8B711C
:10227000C0B20C315469A4898442F6D810BD000064
:102280008401002010B509494B6900219A689B8997
:1022900008E00824145F844201DD022010BD491CBF
:1022A000C9B20C328B42F4D8002010BD840100204A
:1022B00030B50A4C1825616980078A680021C00E74
:1022C00006E01368491CAB4303431360C9B20C32E8
:1022D00063699B898B42F4D830BD000084010020E3
:1022E0000948426900209168928909E00B785B07F0
:1022F0009B0F9B0701D500207047401CC0B20C31DA
:102300008242F3D8022070478401002030B50A4B86
:10231000586982680220002109E01468E50703D0AB
:102320006008400010600020491CC9B20C325C6992
:10233000A4898C42F1D830BD8401002010B5094930
:102340004B6900219A689B8908E00824145F844245
:1023500001DD002010BD491CC9B20C328B42F4D8FB
:10236000022010BD8401002010B509494B690021ED
:102370009A689B8908E00824145F844201DB0020EE
:1023800010BD491CC9B20C328B42F4D8022010BDDA
:102390008401002010B50A494C6900214342A089FC
:1023A000A26808E00824145F9C4201DC002010BDF4
:1023B000491CC9B20C328842F4D8022010BD00007A
:1023C0008401002038B5FFF78BFF284C0028606996
:1023D00022D0406801218078FFF7C6FF002860699D
:1023E00026D0406800214078FFF74CFF00282ED00F
:1023F0001F488079811E3E290DD261696A460968AD
:1024000009798906890E1170694600F0B9F900282A
:1024100001D100F087F838BD41680068497AC17081
:1024200060690029006801D010211AE00D2118E030
:1024300041680068C979C17060690029006801D0ED
:102440000B210EE00A210170FFF74AFC38BD6069DC
:1024500041680068097AC17060690029006802D08B
:102460000321017038BD0221FBE700008401002038
:102470008800002010B5FFF733FF294C0028606961
:1024800022D0406801218078FFF76EFF0028606944
:1024900026D0406800210078FFF766FF00286069B9
:1024A0002AD0406801210079FFF774FF00280AD183
:1024B0006169486809684079C870616900280968DD
:1024C0002AD00120087010BD41680068497AC170A7
:1024D00060690029006801D00F2116E00D2114E089
:1024E00041680068C979C17060690029006801D03D
:1024F0000B210AE00A210BE0416800688979C1706C
:1025000060690029006802D00721017010BD062112
:102510000170FFF7E5FB10BD002000F003F810BDCF
:102520008401002030B5134C05466169002009681C
:1025300040220870606900684168114341600320CF
:10254000FFF7B6FE0C490D4A8888042805D01028EC
:1025500005D008208880032002E0022000E004204B
:1025600010810879616940190968C870FFF776FE23
:1025700030BD00008401002088000020A000002061
:1025800038B5FFF7ADFE304C002860691AD04068BE
:102590000121C078FFF7D2FE00281FD0606900211A
:1025A00040684078FFF7CAFE00283CD0616948685F
:1025B0000968007AC87061690028096842D005205E
:1025C000087038BD41680068497AC17060690029A7
:1025D000006801D0122130E00D212EE0E0681B4D93
:1025E0000078202819D0222817D0E8688068804712
:1025F000002815D0A879811E3E29E2D261696A4679
:10260000096809798906890E1170694600F0B8F8E1
:102610000028D6D1FFF786FF38BD6069006AE5E77C
:10262000FFF75EFB38BD6069416800688979C17059
:1026300060690029006802D00921017038BD0621B7
:102640000170EDE70220BBE7840100208800002034
:10265000F8B500270668044607723D461FE030467D
:1026600000F052F83078202801D0222814D10E48EA
:102670004069006A006880470B484069006800793B
:10268000400601D50120207207484069C1690068F1
:102690000078C000085C07436D1CEDB20836A088C6
:1026A000A842DCD8E780F8BD84010020F8B50027F7
:1026B0000668044607723D461FE0304600F024F8E5
:1026C0003078202801D0222814D10E484069006AB1
:1026D000406880470B48406900680079400601D592
:1026E0000120207207484069C16900680078C00075
:1026F000085C07436D1CEDB20836A088A842DCD800
:10270000E780F8BD840100200649C8600278202ACD
:1027100005D0212A03D0222A01D0232A01D14068E2
:10272000486170478401002070B5134A1369022480
:10273000A3431361114B00281B8805D00D889D42CF
:102740000D8806D85D1B09E0106920431061022046
:1027500070BD0026F643751BED186D1CADB28542A9
:1027600005D30B80106920431061002070BD1069F3
:1027700020431061012070BD00E000E084010020D2
:1027800070B5134A13690224A3431361114B002847
:102790009B7805D00D789D420D7806D85D1B08E02A
:1027A000106920431061022070BD3F26751BED1893
:1027B0006D1CEDB2854205D30B701069204310618A
:1027C000002070BD106920431061012070BD000021
:1027D00000E000E0840100200A490C4B0888401CFE
:1027E000088009480288521C92B202809A4208D995
:1027F0008A780023521CD2B28A703F2A00D98B708B
:102800000380704784010020AA000020E703000035
:1028100002E008C8121F08C1002AFAD170477047A9
:10282000002001E001C1121F002AFBD1704710B542
:102830002220FDF789FE0320FDF76AFE2020FDF728
:1028400083FE10BDFEB51D4617462420FDF77CFE15
:102850007907B8086C46002908D0B808401C410820
:10286000002668434008029101908BE000276843EE
:10287000400801902FE00898C55D002D23D0002668
:1028800000200321EA07225C02D09208920000E0B7
:102890000A4322546D08401C0428F3D36846C178CB
:1028A00000788001014368464078020168468078DC
:1028B000800002431143C8B2FDF72AFE761CF6B22F
:1028C000022EDDD305E0FF20FDF722FEFF20FDF7FD
:1028D0001FFE01987F1CB842CDD8FEBD0898029912
:1028E000855D701CFDF706FC002929D0002D23D042
:1028F000002700200321EA07225C02D09208920000
:1029000000E00A4322546D08401C0428F3D36846B3
:10291000C17800788001014368464078020168462A
:102920008078800002431143C8B2FDF7F1FD7F1C9F
:10293000FFB2022FDDD323E0FF20FDF7E9FD24E005
:10294000F02D22D000200321EA07225C02D0920859
:10295000920000E00A4322546D08401C0428F3D37F
:102960006946C878097889010843694649780A01A7
:102970006946897889000A431043C0B2FDF7C8FD53
:102980000198761CB042A9D8FEBDFF20F6E71220C0
:102990007047AC207047000070B50024FDF75CFD67
:1029A0001020FDF7D1FD0020FDF7B2FD1120FDF74D
:1029B000CBFD0320FDF7ACFD4420FDF7C5FD002055
:1029C000FDF7A6FD1120FDF7A3FD4520FDF7BCFD99
:1029D0000020FDF79DFDAB20FDF79AFD4E20FDF791
:1029E000B3FD0020FDF794FD4F20FDF7ADFD002065
:1029F000FDF78EFDF020FDF7A7FD1F20FDF788FDF8
:102A00002120FDF7A1FD0320FDF782FD2C20FDF71D
:102A10009BFDA020FDF77CFD3C20FDF795FD64208B
:102A2000FDF776FD3220FDF78FFD044D285DFDF7A3
:102A30006FFD641CE4B25A2CF8D370BDA02D0008C1
:102A400010B52220FDF780FDC420FDF761FD202098
:102A5000FDF77AFD10BDF8B504461D4616460F4633
:102A60004420FDF771FD3846FDF752FD2846FDF77D
:102A70004FFD4520FDF768FD2046FDF749FD304636
:102A8000FDF746FD4E20FDF75FFD3846FDF740FDA2
:102A90004F20FDF759FD2046FDF73AFDF8BD10B572
:102AA00004462420FDF750FD2046FDF731FD10BD02
:102AB00094B0FDF745FEFDF751FC3348816B0504EA
:102AC00029438163314801680322D2021143016026
:102AD0001020009001200790052040030024099059
:102AE00008940A946846FDF7F1FF002800D0FEE73D
:102AF0000F200E900F9410941194002112940EA8A0
:102B0000FDF792FE002800D0FEE70020FDF758FCFC
:102B10000120FDF755FC1F481D49846222C0012198
:102B20008461090644620160A02141610121090319
:102B300044600161C4607F21C4618160912189008A
:102B400081624900C46201630838FEF7BBFA0028BD
:102B500000D0FEE700F06AF8FF20FDF7F3FA01234A
:102B60000DA20A210020FDF72BFB04238C22032158
:102B70000F20FDF7B7FBFDF707FC00F019F8002860
:102B8000FBD0FEF719FBF8E7001002400070004090
:102B90000040024010010020546F756368536C6957
:102BA00064657220506F736974696F6E0000000075
:102BB00070B51D4C0025A068002806D12079FEF7CD
:102BC000DDFCFEF7A3FD0120A060FEF7B7FD0026A7
:102BD000002808D1002220791146FEF701FD606827
:102BE000A660401C60606068002810D00E486660D7
:102BF0000C30A660FFF75AFD0B480C30FEF7CAFDFB
:102C000009496420FFF790FD002802D001252846DD
:102C100070BD05480C30FEF715FE002801D00325D5
:102C2000F5E70225F3E700006C00002010B503482B
:102C3000FFF70EFD0248FEF789FC10BD780000206A
:102C4000702C0008000000000400000001000000DB
:102C5000020000000002000004000000010000006B
:102C6000400000000200000000000100020000001F
:102C7000442C0008682C00085001002003000000CC
:102C8000440200000700000010000000191C0008AA
:102C900030000000151D0008010000007524000828
:102CA000230000000520000825000000A91F0008DF
:102CB000290000004D20000802000000C523000884
:102CC00022000000B91E000826000000411E000876
:102CD0002A000000311F000804000000A92000089D
:102CE000240000005D1D0008080000008125000888
:102CF000800000006B110008B0000000D51D000826
:102D0000A1000000D51D0008A2000000D51D00088C
:102D1000A4000000D51D0008A8000000D51D000873
:102D2000400000006D1100089D2100080D220008E0
:102D30008519000800010001000100009800002032
:102D4000740100205001002003000000342D000811
:102D5000682D000880008000882C0008282D0008BD
:102D6000200000003C2D00080000A0FFA000200073
:102D7000000060FF20FF60000000000000FA00007B
:102D800000F4010000E8030000D0070040420F00FB
:102D900080841E0000093D00050001001000200095
:102DA00082000000AA000000AAAA0000AAAAAA00A5
:102DB00055AAAA0055555555AAAAAAAA555555551A
:102DC000AAAAAAAA151515150505050501010101EF
:102DD00000000000000000000000000000000000F3
:102DE00000000000000000000000000000000000E3
:102DF0004145F1FF5F5501000000FFFFFFFFFFFFAE
:102E0000FFFFFFFFFFFFFFFFFFFFFFFFFFFFFFFFD2
:102E1000FFFFFFFFFFFFFFFFFFFFFFFFFFFFFFFFC2
:102E2000FFFFFFFFFFFFFFFFFFFFFFFFFFFFFFFFB2
:102E3000FFFFFFFFFFFFFFCC0003FFCC0003FFFFFE
:102E4000FFFFFFFFFFFFFFFFFFFFFFFFFFFFFFFF92
:102E5000FFFFFFFFFFFFFFFFFFFFFFFFFFFFFFFF82
:102E6000FF0FFFFFC00FFFFFFF0FFFFFFFFFFFFF81
:102E7000FF0FFFFFC00FFFFFFF0FFFFFFFFFFFFF71
:102E8000FFFFFFFFFFFFFFFF33FFFF0003FFFF0018
:102E90000003FFFF3003FF0003FFFF000003FFFFFD
:102EA0003003FFFF33FFFFFFFFFFFFFFFFFFFFFFC9
:102EB000FFFFFFC0FC0FFFC0F003FFCFC0F3FC0F0C
:102EC000C3F0FFCF03F3FFC00F03FFF03F03FFFF8B
:102ED000FFFFFFFFFFFFFFFFFFFFFFFFFFFFFFFF02
:102EE0003F0FFFFF0CF3FFFFCCF3FFFFC30FFFF01B
:102EF000C3FFFFCF33FFFFCF30FFFFF0FCFFFFFF2B
:102F0000FFFFFFFFFFFFFFFFFFFFFFF0FFFFFFC01F
:102F1000303FFFCF000FFFCC0FCFFFF0FFCFFFC040
:102F20003FCFFFCF3FCFFFFFFFFFFFFFFFFFFFFFC1
:102F3000FFFFFFFFFFFFFFFFFFFFFFFFFFFFFFFFA1
:102F4000FFFFFFFFFF0FFFFFC00FFFFFFF0FFFFFA0
:102F5000FFFFFFFFFFFFFFFFFFFFFFFFFFFFFFFF81
:102F6000FFFFFFFFFFFFFFFFFFFFFFF000FFFFC0BE
:102F7000003FFC03FC03FC3FFFC3FFFFFFFFFFFF1D
:102F8000FFFFFFFFFFFFFFFFFFFFFFFFFFFFFFFF51
:102F9000FFFFFC3FFFC3FC03FC03FFC0003FFFF04B
:102FA00000FFFFFFFFFFFFFFFFFFFFFFFFFFFFFF30
:102FB000FFFFFFFFFFFFFFFFFFFFFFFFFC3FFFFFE4
:102FC0000C3FFFFF003FFFFFF003FFFFF003FFFF99
:102FD000003FFFFF0C3FFFFFFC3FFFFFFFFFFFFF36
:102FE000FFFFFFFFFFFFFFFFCFFFFFFFCFFFFFFF51
:102FF000CFFFFFF0003FFFFFCFFFFFFFCFFFFFFF3F
:10300000CFFFFFFFFFFFFFFFFFFFFFFFFFFFFFFF00
:10301000FFFFFFFFFFFFFFFFFFFFF03FFFFFFF038B
:10302000FFFFFFF3FFFFFFFFFFFFFFFFFFFFFFFFBC
:10303000FFFFFFFFFFFFFFFFFFFFFFFFFFFFFFFFA0
:10304000CFFFFFFFCFFFFFFFCFFFFFFFCFFFFFFF50
:10305000CFFFFFFFCFFFFFFFCFFFFFFFFFFFFFFF10
:10306000FFFFFFFFFFFFFFFFFFFFFFFFFFFFFFFF70
:10307000FFFFFFC3FFFFFFC3FFFFFFFFFFFFFFFFD8
:10308000FFFFFFFFFFFFFFFFFFFFFFFFFFFFFFFF50
:10309000FFFFFFFFFFFFFC3FFFFFFC03FFFFFFC041
:1030A0003FFFFFFC0FFFFFFFC0FFFFFFF00FFFFF21
:1030B000FF00FFFFFFF0FFFFFFFFFFFFFFFFFFFF2E
:1030C000FFFFFFFC003FFFF0000FFFC3FFC3FFCF78
:1030D000FFF3FFC3FFC3FFF0000FFFFC003FFFFF44
:1030E000FFFFFFFFFFFFFFFFFFFFFFFFFFFFFFCF20
:1030F000FFCFFFCFFFCFFFCFFFCFFFC00003FFC049
:103100000003FFCFFFFFFFCFFFFFFFCFFFFFFFFF5A
:10311000FFFFFFFFFFFFFFFFFFFFFFC3FC3FFFC0FD
:10312000FC0FFFCC3FC3FFCF0FF3FFCFC3F3FFCFA5
:10313000F003FFCFFC0FFFFFFFFFFFFFFFFFFFFFCD
:10314000FFFFFFF3FFCFFFC3FFC3FFCFF3F3FFCFBB
:10315000F3F3FFCFF3F3FFCFC0F3FFC00003FFF0A3
:103160000F0FFFFFFFFFFFFFFFFFFFFFFFFFFFFF4F
:10317000FFFFFFFC3FFFFFFC03FFFFCCF03FFFCC56
:10318000FF03FFC00003FFC00003FFCCFFFFFFFFF2
:10319000FFFFFFFFFFFFFFFFFFFFFFFFFFFFFFF34B
:1031A000FFFFFFCFC003FFCFF003FFCFF3F3FFCF4D
:1031B000F3F3FFC003F3FFF00FF3FFFFFFFFFFFF89
:1031C000FFFFFFFFFFFFFFFFFFFFFFFC00FFFFF020
:1031D000003FFFC3CF0FFFCFF3C3FFCFF3F3FFC019
:1031E00003F3FFF00FF3FFFFFFFFFFFFFFFFFFFF02
:1031F000FFFFFFFFFFFFFFFFFFC3FFFFFFF3FFFF27
:10320000FFF3FFC0FFF3FFC000F3FFFF0003FFFF6A
:10321000FF03FFFFFFFFFFFFFFFFFFFFFFFFFFFFBA
:10322000FFFFFFF00C0FFFC00003FFCFF3F3FFCF52
:10323000F3F3FFCFF3F3FFC00003FFF00C0FFFFF2A
:10324000FFFFFFFFFFFFFFFFFFFFFFFFFFFFFFCFBE
:10325000F00FFFCFC003FFCFCFF3FFC3CFF3FFF0DB
:10326000F3C3FFF0000FFFFF003FFFFFFFFFFFFF73
:10327000FFFFFFFFFFFFFFFFFFFFFFFFFFFFFFFF5E
:10328000FFFFFFC3F0FFFFC3F0FFFFFFFFFFFFFFE4
:10329000FFFFFFFFFFFFFFFFFFFFFFFFFFFFFFFF3E
:1032A000FFFFFFFFFFFFFFFFFFFFFFFFFFFFFC3FF1
:1032B000FFFFFFC3FFFFFFF3F0FFFFFFF0FFFFFF84
:1032C000FFFFFFFFFFFFFFFFFFFFFFFFFFFFFFFF0E
:1032D000CFFFFFFFCFFFFFFF33FFFFFF33FFFFFCF9
:1032E000FCFFFFF3FF3FFFF3FF3FFFCFFFCFFFCF19
:1032F000FFCFFFFFFFFFFFFFFFFFFFFFFFFFFFFF0E
:1033000033FFFFFF33FFFFFF33FFFFFF33FFFFFFFD
:1033100033FFFFFF33FFFFFF33FFFFFFFFFFFFFF21
:10332000FFFFFFFFFFFFFFCFFFCFFFCFFFCFFFF379
:10333000FF3FFFF3FF3FFFFCFCFFFFFF33FFFFFFFB
:1033400033FFFFFFCFFFFFFFCFFFFFFFFFFFFFFFB9
:10335000FFFFFFFFFFFFFFFFFC3FFFFFFC0FFFCC66
:103360003FCFFFCC0FCFFFFFCFCFFFFFC00FFFFF3F
:10337000F03FFFFFFFFFFFFFFFFFFFFFFFFFFFFF2C
:10338000FFFFFFF0003FFFCFFFCFFF3F0FF3FF3CFA
:10339000F3F3FF3CF3F3FFCC000FFFFFFFFFFFFF52
:1033A000FFFFFFFFFFFFFFFFFFFFFFCFFFFFFFC09C
:1033B000FFCFFFC003CFFFCF000FFFFF3F0FFFFF87
:1033C0003F0FFFCF000FFFC003FFFFC0FFFFFFCF86
:1033D000FFFFFFFFFFFFFFCFFFCFFFC0000FFFC0CA
:1033E000000FFFCFCFCFFFCFCFCFFFCFCFCFFFC0CB
:1033F000000FFFF0303FFFFFFFFFFFFFFFFFFFFF6A
:10340000FFFFFFFC00FFFFF0003FFFC3FF0FFFCFF8
:10341000FFCFFFCFFFCFFFCFFFCFFFCFFFCFFFF318
:10342000FF3FFFFCFC0FFFFFFFFFFFFFFFFFFFCF92
:10343000FFCFFFC0000FFFC0000FFFCFFFCFFFCFB8
:10344000FFCFFFCFFFCFFFC3FF0FFFF0003FFFFC19
:1034500000FFFFFFFFFFFFFFFFFFFFCFFFCFFFC01A
:10346000000FFFC0000FFFCFCFCFFFCFCFCFFFCFD9
:1034700003CFFFCFFFCFFFC0FC0FFFFFFFFFFFFF1A
:10348000FFFFFFFFFFFFFFCFFFCFFFC0000FFFC019
:10349000000FFFCFCFCFFFCFCFCFFFFF03CFFFFF77
:1034A000FFCFFFFFFC0FFFFFFFFFFFFFFFFFFFFF4F
:1034B000FFFFFFFC00FFFFF0003FFFC3FF0FFFCF48
:1034C000FFCFFFCF3FCFFFCF3FCFFFC03F3FFFC07A
:1034D0003C0FFFFF3FFFFFFFFFFFFFFFFFFFFFCF9F
:1034E000FFCFFFC0000FFFC0000FFFCFCFCFFFFF08
:1034F000CFFFFFCFCFCFFFC0000FFFC0000FFFCF28
:10350000FFCFFFFFFFFFFFFFFFFFFFFFFFFFFFCF2B
:10351000FFCFFFCFFFCFFFCFFFCFFFC0000FFFC018
:10352000000FFFCFFFCFFFCFFFCFFFCFFFCFFFFFBA
:10353000FFFFFFFFFFFFFFF03FFFFFC03FFFFFCF99
:10354000FFCFFFCFFFCFFFCFFFCFFFC0000FFFF0B8
:10355000000FFFFFFFCFFFFFFFCFFFFFFFFFFFFFCA
:10356000FFFFFFCFFFCFFFC0000FFFC0000FFFCF57
:103570000FCFFFFF03FFFFFC30CFFFC0FC0FFFC3E7
:10358000FF0FFFCFFFCFFFFFFFFFFFFFFFFFFFCFCB
:10359000FFCFFFCFFFCFFFC0000FFFC0000FFFCF57
:1035A000FFCFFFCFFFCFFFCFFFFFFFCFFFFFFFC05A
:1035B0003FFFFFFFFFFFFFCFFFCFFFC0000FFFC0A8
:1035C000000FFFCFF0FFFFCF03FFFFFC3FFFFFCF58
:1035D00003FFFFCFF0FFFFC0000FFFC0000FFFCFC2
:1035E000FFCFFFFFFFFFFFCFFFCFFFC0000FFFC0E8
:1035F000000FFFCFF0FFFFFF03FFFFFC3FCFFFC037
:10360000000FFFC0000FFFFFFFCFFFFFFFFFFFFF17
:10361000FFFFFFFC00FFFFF0003FFFC3FF0FFFCFE6
:10362000FFCFFFCFFFCFFFCFFFCFFFC3FF0FFFF0D5
:10363000003FFFFC00FFFFFFFFFFFFFFFFFFFFCF8B
:10364000FFCFFFC0000FFFC0000FFFCF3FCFFFCF66
:103650003FCFFFCF3FCFFFFF000FFFFFC03FFFFF78
:10366000FFFFFFFFFFFFFFFFFFFFFFFC00FFFFF07B
:10367000003FFCC3FF0FFC0FFFCFFC0FFFCFFCCFC1
:10368000FFCFFCC3FF0FFC30003FFF3C00FFFFFFFC
:10369000FFFFFFFFFFFFFFCFFFCFFFC0000FFFC007
:1036A000000FFFCFCFCFFFCFCFCFFFFF0FCFFFF068
:1036B000300FFFC0F03FFFCFFFFFFFCFFFFFFFFF47
:1036C000FFFFFFFFFFFFFFC0F03FFFC0C00FFFCFB6
:1036D000C3CFFFCFCFCFFFCF0FCFFFC00C0FFFF077
:1036E0003C0FFFFFFFFFFFFFFFFFFFFFFFFFFFFF9D
:1036F000F00FFFCFFFCFFFCFFFCFFFC0000FFFC006
:10370000000FFFCFFFCFFFCFFFCFFFFFF00FFFFF77
:10371000FFFFFFFFFFFFFFFFFFFFFFFFFFCFFFF0F8
:10372000000FFFF0000FFFCFFFCFFFCFFFFFFFCF56
:10373000FFCFFFF0000FFFF0000FFFFFFFCFFFFFF5
:10374000FFFFFFFFFFFFFFFFFFCFFFFFFC0FFFFFAC
:10375000000FFFC003CFFFC3FFFFFFC003CFFFFF7A
:10376000000FFFFFFC0FFFFFFFCFFFFFFFFFFFFF7B
:10377000FFCFFFFFC00FFFC0000FFFC0FFCFFFF064
:1037800003CFFFFFC0FFFFF003CFFFC0FFCFFFC09D
:10379000000FFFFFC00FFFFFFFCFFFFFFFFFFFCFB7
:1037A000FFCFFFC3FF0FFFC0FC0FFFCC00CFFFFF19
:1037B00003FFFFCC00CFFFC0FC0FFFC3FF0FFFCF05
:1037C000FFCFFFFFFFFFFFFFFFFFFFFFFFCFFFFF69
:1037D000FF0FFFCFFC0FFFCFF0CFFFC003FFFFC0F5
:1037E00003FFFFCFF0CFFFCFFC0FFFFFFF0FFFFF67
:1037F000FFCFFFFFFFFFFFFFFFFFFFC3FC0FFFC077
:10380000FFCFFFCC3FCFFFCF03CFFFCFF0CFFFCF16
:10381000FC0FFFC0FF0FFFFFFFFFFFFFFFFFFFFFDA
:10382000FFFFFFFFFFFFFFFFFFFFFFFFFFFFFFFFA8
:10383000FFFFFC000003FC000003FCFFFFF3FCFFA4
:10384000FFF3FFFFFFFFFFFFFFFFFFFFFFFFFFFF94
:10385000FFFFFFFFFFF0FFFFFF00FFFFF00FFFFF85
:10386000C0FFFFFC0FFFFFC03FFFFC03FFFFFC3F5B
:10387000FFFFFFFFFFFFFFFFFFFFFFFFFFFFFFFF58
:10388000FFFFFCFFFFF3FCFFFFF3FC000003FC0065
:103890000003FFFFFFFFFFFFFFFFFFFFFFFFFFFF33
:1038A000FFFFFFFFFFFFFFFFFFFFFFFFF0FFFFFF37
:1038B000FF3FFFFFFFC3FFFFFFFCFFFFFFC3FFFF53
:1038C000FF3FFFFFF0FFFFFFFFFFFFFFFFFF3FFF97
:1038D000FFFF3FFFFFFF3FFFFFFF3FFFFFFF3FFFF8
:1038E000FFFF3FFFFFFF3FFFFFFF3FFFFFFF3FFFE8
:1038F000FFFF3FFFFFFF3FFFFFFFFFFFFFFFFFFF58
:10390000FFFFFFFFFFFFFFFFFFFFFFFFFFFCFFFFCA
:10391000FFF3FFFFFFCFFFFFFFFFFFFFFFFFFFFFF3
:10392000FFFFFFFFFFFFFFFFFFFFFFFFFFFFFFF0B6
:10393000FFFFFFC03CFFFFCF3CFFFFCF3CFFFFF38B
:103940003CFFFFC000FFFFC003FFFFCFFFFFFFFFF3
:10395000FFFFFFFFFFFFFFCFFFF3FFC00003FFC02C
:103960000003FFF3F3FFFFCFFCFFFFCFFCFFFFC31C
:10397000F0FFFFF003FFFFFC0FFFFFFFFFFFFFFF64
:10398000FFFFFFFC0FFFFFF003FFFFC3F0FFFFCFC0
:10399000FCFFFFCFFCFFFFCFFCFFFFC3F3FFFFF0F7
:1039A000C0FFFFFFFFFFFFFFFFFFFFFFFFFFFFFC69
:1039B0000FFFFFF003FFFFC3F0FFFFCFFCFFFFCFC0
:1039C000FCFFFFF3F3F3FFC00003FFC00003FFCFD2
:1039D000FFFFFFFFFFFFFFFFFFFFFFFC0FFFFFF0F9
:1039E00003FFFFC330FFFFCF3CFFFFCF3CFFFFCF04
:1039F00030FFFFC303FFFFF30FFFFFFFFFFFFFFFDA
:103A0000FFFFFFFFFFFFFFFFFFFFFFCFFCFFFFCF29
:103A1000FCFFFFC0000FFFC00003FFCFFCF3FFCF90
:103A2000FCF3FFCFFCF3FFFFFFF3FFFFFFF3FFFF0C
:103A3000FFFFFFFC0FFFFFF003FFF3C3F0FFF3CF27
:103A4000FCFFF3CFFCFFF3F3F3FFF00000FFFC00FB
:103A500000FFFFFFFCFFFFFFFFFFFFFFFFFFFFCFA8
:103A6000FFF3FFC00003FFC00003FFCFF3FFFFFF22
:103A7000FCFFFFCFFCFFFFC000FFFFC003FFFFCF35
:103A8000FFFFFFFFFFFFFFFFFFFFFFFFFFFFFFCF76
:103A9000FFFFFFCFFCFFFFCFFCFFFFC000C3FFC055
:103AA00000C3FFCFFFFFFFCFFFFFFFCFFFFFFFFFF1
:103AB000FFFFFFFFFFFFFFFFFFFFF3FFFCFFF3FF31
:103AC000FCFFF3FFFCFFF3FFFCC3F00000C3FC00AE
:103AD00000FFFFFFFFFFFFFFFFFFFFFFFFFFFFFFF5
:103AE000FFFFFFCFFFF3FFC00003FFC00003FFFF96
:103AF0000FFFFFCC00FFFFC0F0FFFFC3FCFFFFCFB5
:103B0000FCFFFFCFFFFFFFFFFFFFFFFFFFFFFFCF28
:103B1000FFFFFFCFFFF3FFCFFFF3FFC00003FFC0A6
:103B20000003FFCFFFFFFFCFFFFFFFCFFFFFFFFF30
:103B3000FFFFFFFFFFFFFFFFFFFFFFCFFCFFFFC007
:103B400000FFFFC000FFFFFFFCFFFFC000FFFFC042
:103B500000FFFFFFFCFFFFC000FFFFC003FFFFCF20
:103B6000FFFFFFFFFFFFFFCFFCFFFFC000FFFFC015
:103B700000FFFFCFF3FFFFFFFCFFFFCFFCFFFFC005
:103B800000FFFFC003FFFFCFFFFFFFFFFFFFFFFFAF
:103B9000FFFFFFFC0FFFFFF003FFFFC3F0FFFFCFAE
:103BA000FCFFFFCFFCFFFFCFFCFFFFC3F0FFFFF0E8
:103BB00003FFFFFC0FFFFFFFFFFFFFFFFFFFF3FF10
:103BC000FCFFF00000FFF00000FFF3F3F3FFF3CF82
:103BD000FCFFFFCFFCFFFFC3F0FFFFF003FFFFFC84
:103BE0000FFFFFFFFFFFFFFFFFFFFFFC0FFFFFF0D7
:103BF00003FFFFC3F0FFFFCFFCFFF3CFFCFFF3F3A6
:103C0000F3FFF00000FFF00000FFF3FFFCFFFFFFF9
:103C1000FFFFFFFFFFFFFFCFFCFFFFCFFCFFFFC059
:103C200000FFFFC000FFFFCFF3FFFFCFFCFFFFCF80
:103C3000FCFFFFFFF0FFFFFFF3FFFFFFFFFFFFFFB2
:103C4000FFFFFFC3C3FFFFC300FFFFCF0CFFFFCF8A
:103C50000CFFFFCC3CFFFFC030FFFFF0F0FFFFFF89
:103C6000FFFFFFFFFFFFFFFFFFFFFFFFFFFFFFFF64
:103C7000FCFFFFFFFCFFFFF00003FFC00003FFCFCE
:103C8000FCFFFFCFFCFFFFCFFCFFFFF3FFFFFFFFB9
:103C9000FFFFFFFFFFFFFFFFFFFFFFFFFCFFFFF046
:103CA00000FFFFC000FFFFCFFFFFFFCFFFFFFFF3CD
:103CB000FCFFFFC000FFFFC000FFFFCFFFFFFFFFC3
:103CC000FFFFFFFFFFFFFFFFFCFFFFFFC0FFFFFC49
:103CD00000FFFFC03CFFFFC3FFFFFFC03CFFFFFC36
:103CE00000FFFFFFC0FFFFFFFCFFFFFFFFFFFFFF25
:103CF000FCFFFFFF00FFFFC000FFFFC0FCFFFFF065
:103D00003FFFFFFF0FFFFFF03FFFFFC0FCFFFFC0C3
:103D100000FFFFFF00FFFFFFFCFFFFFFFFFFFFCFE4
:103D2000FCFFFFCFFCFFFFC3F0FFFFC000FFFFFC65
:103D30000FFFFFC000FFFFC3F0FFFFCFFCFFFFCF6F
:103D4000FCFFFFFFFFFFFFFFFFFFFFFFFCFFF3FF95
:103D5000F0FFF3FF00FFF0F00CFFF003FFFFF300B4
:103D6000FFFFFFF00CFFFFFF00FFFFFFF0FFFFFF73
:103D7000FCFFFFFFFFFFFFFFFFFFFFC3F0FFFFC0E0
:103D8000FCFFFFCC3CFFFFCF3CFFFFCF0CFFFFCF82
:103D9000C0FFFFC3F0FFFFFFFFFFFFFFFFFFFFFFBD
:103DA000FFFFFFFFFFFFFFFFFFFFFFFF3FFFFF00E2
:103DB000000FFC00C003FCFFFFF3FFFFFFFFFFFF4E
:103DC000FFFFFFFFFFFFFFFFFFFFFFFFFFFFFFFF03
:103DD000FFFFFFFFFFFFFFFFFFFFFFFFFFFFFC00F5
:103DE0000003FC000003FFFFFFFFFFFFFFFFFFFFDB
:103DF000FFFFFFFFFFFFFFFFFFFFFFFFFFFFFFFFD3
:103E0000FFFFFFFFFFFFFCFFFFF3FC00C003FF000D
:103E1000000FFFFF3FFFFFFFFFFFFFFFFFFFFFFF61
:103E2000FFFFFFFFFFFFFFFFFFFFFFFFCFFFFFFFD2
:103E3000F3FFFFFFF3FFFFFFCFFFFFFF3FFFFFFF9A
:103E40003FFFFFFFCFFFFFFFFFFFFFFFFFFFFFFF72
:103E5000FFFFFFFFFFFFFFFFFFFFFFFFFFFFFFFF72
:103E6000FFFFFFFFFFFFFFFFFFFFFFFFFCF003FF70
:103E7000FFFFFFFFFFFFFFFFFCF003FCF003FCF080
:103E800003FCF003FCF003FCF003FCF003FFFFFF76
:103E9000F0CCFFFF003FF0CCC3FF003FF0CCC3FFEE
:103EA000FFFFFFFFFFFF0C3FFF33CFF033C3FFC324
:103EB000CFFFFFFFFFFFFFFFFFFFFFF3CFFFF33356
:103EC000FF33CFFCCCFFFF3CFFFFFFFFFFFFFFFFF7
:103ED0000FFFFCF0FFFCCF3FFF3F3FFCCFFFFFFF9A
:103EE000FFFFFFFFFFFFFFFFFFFFFFFCF3FFFFFFF1
:103EF000FFFFFFFFFFFFFFFFFFFFFFFFFFFFFFFCD5
:103F0000FF3FC3FFC3FFFFFFFFFFFFFFFFFFFFFFF9
:103F1000FFC3FFC3FCFF3FFFFFFFFFFFFFFFFFFFEC
:103F2000FFFFFFFFFFCFFFF0CFFFFF03FFF0CFFF4B
:103F3000FFCFFFFFFFFFF3FFFFF3FFFFF3FFFC00E7
:103F40000FFFF3FFFFF3FFFFF3FFFFFFFFFFFFFF95
:103F5000C3FFFFF03FFFFF3FFFFFFFFFFFFFFFFF3C
:103F6000FFFFFFF3FFFFF3FFFFF3FFFFF3FFFFF39D
:103F7000FFFFFFFFFFFFFFFFFFFFFC3FFFFC3FFFD7
:103F8000FFFFFFFFFFFFFFFFFFFFFFFFF3FFFFFC50
:103F90003FFFFFC3FFFFFC3FFFFFC3FFFFFFFFFF2C
:103FA000FFFF000FFCFFF3FCFFF3FCFFF3FF000F2C
:103FB000FFFFFFFFFFFFFCFFFFFCFFF3FC0003FC24
:103FC000FFFFFCFFFFFFFFFFFFFFFFFC3FCFFCCF2A
:103FD000F3FCF3F3FCFCF3FC3F0FFFFFFFFFFFFFDD
:103FE000FF3FCFFCFFF3FCFCF3FCFCF3FF030FFFF0
:103FF000FFFFFFFFFFFFC3FFFFCCFFFFCF0FFCCF93
:10400000F3FC0003FCCFFFFFFFFFFF3FFFFCFC03BF
:10401000FCFCF3FCFCF3FF03F3FFFFFFFFFFFFFFDC
:10402000003FFCFCCFFCFCF3FCFCF3FF03F3FFFFC1
:10403000FFFFFFFFFFFFC3FFFFF3FC3FF3FFC0F3F2
:10404000FFFF03FFFFFFFFFFFFFF030FFCFCF3FC7D
:10405000FCF3FCFCF3FF030FFFFFFFFFFFFFFCFC83
:104060000FFCF3F3FCF3F3FF33F3FFC00FFFFFFF8D
:10407000FFFFFFFFFFFFFC3C3FFC3C3FFFFFFFFF5C
:10408000FFFFFFFFFFFFFFFFFFFFFFF0FFFFFC3C15
:10409000CFFF3CCFFFFFFFFFFFFFFFF3FFFFCCFF92
:1040A000FFCCFFFF3F3FFCFFCFFCFFCFFFFFFFFF39
:1040B000FFFFFFCCFFFFCCFFFFCCFFFFCCFFFFCC0F
:1040C000FFFFFFFFFCFFCFFCFFCFFF3F3FFFCCFF19
:1040D000FFCCFFFFF3FFFFFFFFFFFFFFFFFFFFFC32
:1040E000FF3FFCFFCFFFF3CFFFFC3FFFFFFFFFFFD2
:1040F000FFFC0003F3FFFCF3F0FCF3CF3CFCC00338
:10410000FFFFFFFCFFFFFC0FFFFCC033FFCFC3FC32
:10411000C03FFC0FFFFCFFFFFCFFF3FC0003FCFCB7
:10412000F3FCFCF3FCFCF3FF030FFFFFFFFFFFFFBB
:10413000FF000FFCFFF3FCFFF3FCFFF3FF3FC3FFA7
:10414000FFFFFCFFF3FC0003FCFFF3FCFFF3FF3F6A
:10415000CFFFC03FFFFFFFFCFFF3FC0003FCFCF3BD
:10416000FCF033FCFFF3FC3FC3FFFFFFFFFFFFFC4E
:10417000FFF3FC0003FCFCF3FFF033FFFFF3FFFF52
:10418000C3FFFFFFFF000FFCFFF3FCF3F3FF03C3CC
:10419000FFF3FFFFFFFFFCFFF3FC0003FCFCF3FF5A
:1041A000FCFFFCFCF3FC0003FCFFF3FFFFFFFCFF44
:1041B000F3FCFFF3FC0003FCFFF3FCFFF3FFFFFF46
:1041C000FFFFFFFF03FFFCFFF3FCFFF3FF0003FF14
:1041D000FFF3FFFFFFFCFFF3FC0003FCF3F3FFF032
:1041E000FFFFCF33FC3FC3FCFFF3FFFFFFFCFFF3F8
:1041F000FC0003FCFFF3FCFFFFFC0FFFFFFFFFFCD5
:10420000FFF3FC0003FCFF03FFF0FFFCFF03FC00D7
:1042100003FCFFF3FCFFF3FC0003FCFF03FFC0FF04
:10422000FC3FF3FC0003FFFFF3FFFFFFFF000FFC69
:10423000FFF3FCFFF3FCFFF3FF000FFFFFFFFFFFA7
:10424000FFFCFFF3FC0003FCF3F3FFF3F3FFFC0FB1
:10425000FFFFFFFFFFFFFF000FFCFFF3F0FFF3F096
:10426000FFF3F3000FFFFFFFFCFFF3FC0003FCF381
:10427000F3FFF3F3FFC3F3FF3C0FFCFFFFFFFFFF70
:10428000FC3F0FFF3CF3FCFCF3FCFCCFFF03C3FF40
:10429000FFFFFFFFC3FFFFF3FCFFF3FC0003FCFF86
:1042A000F3FFFFF3FFFFC3FFFFF3FF0003FCFFF388
:1042B000FCFFFFFCFFF3FF0003FFFFF3FFFFF3FF33
:1042C000FF03FFC0F3FC3FFFFFC0F3FFFF03FFFF4F
:1042D000F3FFFFF3FF0003FCFFF3FF00FFFCFFF31E
:1042E000FF0003FFFFF3FCFFF3FC3FC3FFCF3FFFE3
:1042F000F0FFFFCF3FFC3FC3FCFFF3FFFFF3FFFFE7
:10430000C3FCFC33FC03FFFCFC33FFFFC3FFFFF3E4
:10431000FFFFFFFC3FC3FCCFF3FCF0F3FCFF33FCDB
:104320003FC3FFFFFFFFFFFFFFFFFFC00003CFFF03
:10433000F3CFFFF3FFFFFFFFFFFFFFFFFFFFFFF3E1
:10434000FFFC0FFFC3FFF03FFFFFFFFFFFFFFFFF7B
:10435000FFFFFFFFFFCFFFF3CFFFF3C00003FFFF1F
:10436000FFFFFFFFFFFFFFFFFCFFFFFF3FFFFFC35C
:10437000FFFF3FFFFCFFFFFFFF3FFFFF3FFFFF3F50
:10438000FFFF3FFFFF3FFFFF3FFFFF3FFFFFFFFF3D
:10439000FFFFFFFFFFFFFFFFFFF3FFFFCFFFFFFF69
:1043A000FFFFFFFFFFFFFF0CFFFCF33FFCF33FFCB1
:1043B000F33FFC00FFFCFFFFFCFFF3FC0003FCFCF1
:1043C000FFFCFF3FFCFF3FFF00FFFFFFFFFFFFFF82
:1043D000FF00FFFCFF3FFCFF3FFCFF3FFF3C3FFFB8
:1043E000FFFFFFFFFFFF00FFFCFF3FFCFF3FFCFC68
:1043F000F3FC0003FCFFFFFFFFFFFF00FFFCF33FA8
:10440000FCF33FFCF33FFCF0FFFFFFFFFFFFFFFC6F
:10441000FF3FFC000FFCFF33FCFF33FCFF33FFFFCB
:10442000FFFFFFFFFF00FFCCFF3FCCFF3FCCFCFFB7
:10443000F0003FFFFF3FFCFFF3FC0003FCFCFFFF2D
:10444000FF3FFCFF3FFC00FFFCFFFFFFFFFFFCFF07
:104450003FFCFF3FFC0033FCFFFFFCFFFFFFFFFFC3
:10446000FFFFFFCFFF3FCFFF3FCFFF33F0003FFF06
:10447000FFFFFFFFFFFCFFF3FC0003FFF3FFFCC3A4
:104480003FFC3C3FFCFF3FFFFFFFFFFFFFFCFFFF48
:10449000FCFFF3FC0003FCFFFFFCFFFFFFFFFFFC42
:1044A000FF3FFC003FFCFF3FFC00FFFCFF3FFC0028
:1044B000FFFCFFFFFCFF3FFC003FFCFCFFFFFF3F5A
:1044C000FCFF3FFC00FFFCFFFFFFFFFFFF00FFFCC6
:1044D000FF3FFCFF3FFCFF3FFF00FFFFFFFFCFFF61
:1044E0003FC0003FCCFCFFFCFF3FFCFF3FFF00FF55
:1044F000FFFFFFFFFFFFFF00FFFCFF3FFCFF3FCC84
:10450000FCFFC0003FCFFF3FFFFFFFFCFF3FFC0071
:104510003FFCFCFFFCFF3FFCFF3FFFFFFFFFFFFFF7
:10452000FC3CFFFCF33FFCF33FFCF33FFF0C3FFF81
:10453000FFFFFFFFFFFFFF3FFF000FFCFF3FFCFF00
:104540003FFCFF3FFF3FFFFFFF3FFF003FFCFFFF40
:10455000FCFFFFFF3F3FFC003FFCFFFFFFFF3FFF73
:10456000F03FFF0F3FFCFFFFFF0F3FFFF03FFFFF5C
:104570003FFFFF3FFF003FFCFF3FFF03FFFCFF3F0C
:10458000FF003FFFFF3FFCFF3FFC3C3FFFC3FFFF3F
:10459000C3FFFC3C3FFCFF3FFFFFFFFFFF3FCFFCA3
:1045A0003FCFC33FC03FFFCF0F3FFFF03FFFFF3F75
:1045B000FFFFFFFC3C3FFCCF3FFCF33FFCFC3FFC1C
:1045C0003F3FFFFFFFFFFFFFFFFFFFFFCFFFF03089
:1045D0000FCFFFF3FFFFFFFFFFFFFFFFFFFFFFFF17
:1045E000FFFFFFF00003FFFFFFFFFFFFFFFFFFFFE5
:1045F000FFFFFFFFFFCFFFF3F0300FFFCFFFFFFF05
:10460000FFFFFFFFFFFFFFFFCFFFFFF3FFFFCFFF26
:10461000FFCFFFFFF3FFFFFFFF0000003C46000855
:104620000000002010010000102800084C4700087E
:1046300010010020E0040000202800080000000015
:10464000ABAA5555ABAA5555ABAA5555ABAA55556E
:10465000ABAA5555ABAA5555ABAA5555ABAA55555E
:10466000ABAA5555ABAA5555ABAA5555ABAA55554E
:10467000ABAA5555ABAA5555ABAA5555ABAA55553E
:10468000ABAA5555ABAA000080841E0000000000B4
:1046900000000000010203040607080903040608DD
:1046A0000C10182030000000000000000000000086
:1046B00000000000602D0008010000000000000064
:1046C000000000000A00FF1F04000500882C0008FD
:1046D000282D00080000000000000000000000007D
:1046E00000000000000000000000000003040608B5
:1046F0000C10182030000000000102030401020326
:1047000004060708090000000000005000040050E3
:1047100000000050992900089F2A0008572A000825
:10472000412A00082F280008932900088F29000833
:10473000452800080000000000000000FA2D0008D5
:0C4740000B0004004E3E000807000300C0
:04000005080000C12E
:00000001FF
